:020000040000FA
:090000000219FD858A6502040A5B
:03000B000215B02B
:0500130002041601FFCC
:0F001B003034F8B280C574C8868BC804C57432FF
:03002B000203E2EB
:03003B000215307B
:03005B0002042577
:10007300C2AF53E67F7592FA7593FFD2AF53917F68
:0C008300302D08C22D303B0302157032F6
:1000B0004A45534330312023323420202020202051
:1000C0000406080C10182030406080A0C0C2AFC0E9
:1000D00082C083901480E493B4541BA3E493B44C83
:1000E00015A3E493B4580FA3A3A3E493B404071295
:1000F0001500D23B8002C23BD083D082D2AF22C255
:10010000AFC2A8C2CAC28EC0D075D008A8CCA9CD33
:10011000D2CAD2AF53E6EF85618BC0E0C0F0758ADA
:1001200000C3E89562F8E99563F9C3E913F9E813A8
:10013000F8E97021E89573401C95735018E582B476
:1001400010137C007B007A007908900000A860C33F
:10015000E813F8215E900000D2A8D2AA6134E0FD35
:10016000C39CC39840EF98EB33FB0582E0FCC39D32
:10017000C39840E198EB33FB0582E0FDC39CC39834
:1001800040D398EB33FB0582E0FCC39DC39840C588
:1001900098EB33FB0582E0FDC39CC39840B798EB16
:1001A00033FB0582E0FCC39DC39840A998EB33FB69
:1001B0000582E0FDC39CC398409B98EB33FB05820E
:1001C000E0FCC39DC398408D98EB33FB058221D999
:1001D000900000D2A8D2AA6134E0FDC39CC398402D
:1001E000EF98EA33FA0582E0FCC39DC39840E1989A
:1001F000EA33FA0582E0FDC39CC39840D398EA3302
:10020000FA0582E0FCC39DC39840C598EA33FA051D
:1002100082E0FDC39CC39840B798EA33FA0582E0B8
:10022000FCC39DC39840A998EA33FA0582E0FDC358
:100230009CC398409B98EA33FA0582E0FCC39DC3B7
:1002400098408D98EA33FA0582EBC46B6A54F0F952
:10025000EAC4303301F454F0C3996009900000D22D
:10026000A8D2AA6134D2C0EBF4C454F0F9EAF4C4C1
:10027000540F49FAEBF4C4540FFBC3EAF99460FA43
:10028000EB9400FB5020C3E97B007A0079006016F4
:10029000C3135006F9C3954D600AE9F54D754E003C
:1002A00079008002054E303A27C3EA94D0F8EB94E7
:1002B00007F9400BE8FAE9FB203109D23141C4309B
:1002C0003102C231203902B231C3EA33FAEB33FBD7
:1002D000EB2B3B3BF9C3EB13FBEA13FAEA29FAEBEE
:1002E0003400FB30E3047AFF7BFFE5255403601BF9
:1002F000202A18E55833F9EB7007C3E99A4002E960
:10030000FAE536C4332AFAEB3400FBC3EA33C454AB
:100310000FF8EB33C454F048F87005EA6002780136
:10032000900000E52260021522614A900000D2A8E8
:10033000D2AA61340522E52270021522C3E5229477
:1003400032500261BF754F0061C2884FD230E86001
:1003500003755000C3E556FC95574002AC57C3ECFB
:10036000954F5008EC75F008A4FAABF0EBF41313BA
:1003700092D5A2E75401F9EAF4FC13A2D513F8E5EB
:100380006423F564EC54032431835564600BE82442
:1003900001E9340020E10208F9C3E89423FAE99462
:1003A00000FB50047A007B00885189528A538B5499
:1003B00075230A53F7DF43F740800700115577751F
:1003C000230AE5E6A2E082C0400ED2AAD2A8D0F06D
:1003D000D0E0D0D043E6103243E610D0F0D0E0D0E9
:1003E000D032C0D0C0E0C2CF053AE5236002152369
:1003F000C3E54F60057550008105E5502401F550B7
:1004000050037550FFD0E0D0D032C0E0E565856183
:100410008BF0A3D0E032C2AAD28EC2CA85CC62854C
:10042000CD63D2CA3253F7DFC0E0E5F9E5FA30E137
:100430000F8551FB8552FC8553E98554EA53F7BF7C
:10044000D0E0327901801879038014790A8010791C
:100450000F800C791E80087964800479C880007848
:100460001474F0000000D5E0FAD8F6D9F222790130
:10047000801479038010790A800C791E80087964D1
:10048000800479C880007591007594987595FC7505
:100490009104D22D43E680303B0953E67F302D0690
:1004A000121550202DFDD9DE2278FF20282879A1B1
:1004B000E76023E571601F74FF8571F0848539F072
:1004C00030290375F005A4F8C5F0600278FFC3E891
:1004D00095585002A858885722C3E57094E4E571F6
:1004E0009400E55750031481EA046002F557227521
:1004F000E890220559C3E5599408405330EDF4A81B
:10050000BDA9BE755900E9FA79A0E76041EA700615
:10051000E55A6018800CC3E8955A600EE55A5005FC
:10052000600A1480070460FA8002E55AF55AC39500
:100530005F401B7556C0C394044013755680C39426
:1005400004400B755640C39404400375560022E5E1
:10055000562410500274FFF55622743279A687F0A3
:10056000A4C5F0A2F733F558227570007571F0221A
:10057000C2AFC2CAA8CCA9CDAA3A30CF010AD2CA0A
:10058000D2AFC3EA13FAE913F9E813F8853B3E85C5
:100590003C3F883B893C8A3D22C2AFC2CAA8CCA955
:1005A000CDAA3A30CF010AD2CAD2AFAB3BAC3C881D
:1005B0003B893CC3E89BF8E99C202809F9302C03CF
:1005C0000206AC803FAD3D8A3DF9EA9DFA600678AF
:1005D000FF79FF8013AE3EAF3F8B3E8C3FA83BA917
:1005E0003CC3E89EF8E99FF9C3E57113FBE570137E
:1005F000FAE82AF570E93BF57150067570FF7571E0
:10060000FF020651AA70AB71AC70AD717E047F021F
:10061000C3EB9404400D1E1FC3EB94084005202932
:10062000021E1FC3ED13FDEC13FCDEF7C3EA9CFAB8
:10063000EB9DFBEF6009C3E913F9E813F8DFF7EA74
:1006400028FAEB39FB8A708B7150067BFF8B708B1D
:1006500071C3EB94025002D22C3028057F030206AE
:100660007D7892E6FFC3E537948240110FC3E537EA
:1006700094A040010FC3EF940640027F057E02E57F
:1006800071C4540FF9E571C454F0F8E570C4540F07
:1006900028F8C3E89EFAE99400FB4009C3EA9401F4
:1006A000EB940050047A01E4FB0206F8AA70AB71E7
:1006B000EBC4FEEAC4540F4EFCC3EA9CFAEB940070
:1006C000FBC3E813C313F8EA28FAEB3400FB8A7083
:1006D0008B71C3EB94024002C22C7802EBC4FE7B08
:1006E00000EAC4540F4EFAC3EA98FA4005C39401D5
:1006F00050027A017892E6FF303B0953E67F302DB5
:1007000006121550202DFD854992854A93D22D431E
:10071000E680C3E49AF8E49BF9302C03020790E8E2
:10072000FAE9FBD3E913FDE813FC8849894AC3EFD2
:1007300094036038EF20E00CE82CF8E93DF9ECFA7E
:10074000EDFB8013E828F8E939F9C3E82401F8E95A
:100750003400F97AFF7BFFC3EF9403400F8A4B8B81
:100760004C884589468C478D480207C5884B894C83
:100770008A458B468C478D48302812754BF0754C56
:10078000FF7547F07548FF7549F0754AFF0207C5C8
:10079000E8FAD3E813FC8849C3EF94036021EF2003
:1007A000E007E82CF8ECFAE1B0E8282401F87AFF39
:1007B000C3EF940340098A4B88458C470207C588DC
:1007C0004B8A458C47303B0953E67F302D06121586
:1007D00050202DFD753402D22D43E680E5255403CB
:1007E0006034A870A971C3E913F9E813F8C3E913D9
:1007F000F9E813F8302804E92440F9C2AF53E67F42
:10080000759100C3E498F594E499F595759104D237
:100810002D43E680D2AF22D22075440075200030EF
:100820002B03752040800ED2207544007520403087
:100830002B0375200078017901202C20E525540335
:100840006002C2207914E571C313700104F8C394E7
:100850001440027814302804781B791B202D11E5F0
:1008600044600D302803D53404D22101E41207D7A7
:100870000544E59B5440B52004D2A001CCC2A03071
:10088000280908C3E899400118015C20200B08C31F
:10089000E8994003020835015CC22053E67F759158
:1008A00000302C117594007595F8759104D22D4384
:1008B000E680020835E5717EFFC3334005C333404F
:1008C00001FEC3E49E759400F59501AAC3E5339437
:1008D000015003020835302003020835D80201E236
:1008E000015CC221C2A0C2AF53E67F759100854B67
:1008F00094854C95759104854592854693D22D43F8
:10090000E680D2AFE5255403600720290205338035
:100910001030210D202B0A2020071581158102118E
:10092000832278003020027801E53775F007A4F9BA
:10093000E5F028F5F0E9A2F013A2F113A2F213F505
:1009400037C394785003753778C3E5379538400C32
:10095000C286C290C29275D4FF75D50F303B095341
:10096000E67F302D06121550202DFD8547928548D3
:1009700093D22D43E68022203813C2AFC291D28792
:1009800075D4FF75D503D2AF759F42416BC2AFC21C
:1009900091D29375D43F75D50FD2AF759F42416BFD
:1009A000203813C2AFC29275D4FF75D50CD287D24E
:1009B000AF759F52416BC2AFC28675D4FF75D50C1F
:1009C000D293D2AF759F32416B203813C2AFC2872A
:1009D000D29375D4FF75D50CD2AF759F32416BC2DF
:1009E000AFC293D28775D4FF75D50CD2AF759F5225
:1009F0008079203813C2AFC29075D43F75D50FD21D
:100A000093D2AF759F428063C2AFC29075D4FF7519
:100A1000D503D287D2AF759F428050203813C2AF22
:100A2000C293D29175D43F75D50FD2AF759F5280C6
:100A30003AC2AFC287D29175D4FF75D503D2AF75D4
:100A40009F328027203813C2AFC28675D4FF75D578
:100A500003D291D2AF759F328011C2AFC29275D4CA
:100A60003F75D50FD291D2AF759F52227A1C7B3C35
:100A700080127A147B4B800C7A107B5A80067A0A9B
:100A80007B788000E55BD5E001227902E4C291D554
:100A9000E0FDD290D5E0FDC290D5E0FDD291D5E049
:100AA000FDE920E002D28630E002D292E55BD5E09B
:100AB000FDE920E002C28630E002C2927496D5E0E1
:100AC000FDD9C9EAF8D5E0FDD8FBDBB8C29122C256
:100AD00086C290C292C287C291C29375D4FF75D567
:100AE0000F22788076FF0876FF0876FF0876FF08E9
:100AF00076FF0876FF0876090876FF087601788C7D
:100B000076010876FF0876FF0876FF0876FF0876FC
:100B1000FF0876030876FF0876FF0876FF0876253B
:100B20000876D00876280876500876040876FF08FC
:100B300076020876FF08767A0876FF087607087648
:100B4000010876FF0876FF0876000876002278888C
:100B5000E6C39403D23A5002C23AC238E630E10208
:100B6000D238A23892397886E6149000C09378A6DD
:100B7000F67886E6F539C394025003753902789CFD
:100B8000E67538FFB402037538A0B40303753882E4
:100B900078A0E6F8600674282409D8FCF55F22786E
:100BA000A5E6F954037000E9540C7000E954307064
:100BB00000E954C0700022755D00755E007597DE17
:100BC0007597AD7581C043FF8075EF0675A90075F7
:100BD000A90051CF75803F75F1C375A4C075803FE2
:100BE00075D4FF75900075F20F75A50F759000759F
:100BF000D50F75A00075A601E5B525E0600975A7BC
:100C00001075CF0075A70075E34075E20251CFE47F
:100C1000F8F6D8FD51E21211B97898865B7530016B
:100C2000756401C2AF12045B516C12044F12044F81
:100C300012044F517212044F12044F12044F517894
:100C400012044F12044F12044F517E517E1204576A
:100C5000719FC2AF53A4FED280755D00755E00AA7D
:100C6000E475E48078FA79FA308009D9FBD8F70284
:100C70001C008AE4C2AF714E7898865B51CF75C86C
:100C800004759104C22D75D84075D90875F7817522
:100C90009E0375960275DA4275DB4275A82175E6EA
:100CA0001043B805759B80759D0075D10C75BC59B6
:100CB00075BB1075E88075B2011204439000007591
:100CC0008800757201753600C230754D00754E0092
:100CD00075E4081200CDD2337588517589AA758CD8
:100CE00000758D00C2A9D2ABD2AAD2AF758E0175A4
:100CF00061C075601475735075220A1200CD12041C
:100D00007E756010C3E522940A754D00754E004053
:100D100077758E0C75618075602875732875220A49
:100D20001200CD12047E756020C3E522940A754D31
:100D300000754E00405275E480C233758E017561B6
:100D4000C075601475735075220A1200CD12047EAE
:100D5000756010C3E522940A754D00754E00402859
:100D6000758E0C75618075602875732875220A125E
:100D700000CD12047E756020C3E522940A754D00F3
:100D8000754E004003020C52120472203003020C14
:100D900052C2AFA233823B4006517E517E80045145
:100DA000785178D2AF12048212047EC3E54F9401C9
:100DB000400280EFC2AFA233823B401D516CD2AFE4
:100DC00012047EC2AF516CD2AF12047EC2AF516C1E
:100DD000D2AF12047EC2AF8006517E517E517ED2C8
:100DE000AF12048275300075700075710075400097
:100DF000754100E4F531F5327520000520300147DA
:100E00007520000531E531F4703D0532789AE678B9
:100E100019146012783214600D787D14600878FA25
:100E2000146003753200C3E53298401B51CF1204A1
:100E30004315327531007899865BC2AF517ED2AFCF
:100E40007898865B12047E120476E5237002815244
:100E500012046E3030A5C3E54F9401500AC3E54D2E
:100E600094015016020DFB12047EE5237003020C60
:100E700052754D00754E00021023C3E54D9401706C
:100E800016C2AF51CF7899865B516C7898865BD249
:100E9000AF12047E021012C3E54D94027016C2AF69
:100EA00051CF7899865B51727898865BD2AF1204E5
:100EB0007E021012C3E54D94037016C2AF51CF7875
:100EC00099865B51787898865BD2AF12047E0210C7
:100ED00012C3E54D94047016C2AF51CF7899865B6A
:100EE000517E7898865BD2AF12047E021012C3E561
:100EF0004D94057016C2AF51CF7899865B517E78BC
:100F000098865BD2AF12047E021012C3E54D94079F
:100F1000701BC3E54E94065002020E507401303A25
:100F20000274037888F6C238C239021012C3E54D44
:100F30009408701BC3E54E94065002020E507402D2
:100F4000303A0274047888F6D238D239021012C3CB
:100F5000E54D94097019C3E54E94065003020E50F6
:100F6000303A0CC37888E69402F6C23A021012C3F3
:100F7000E54D940A7018C3E54E94065003020E50D6
:100F8000203A0B7888E62402F6D23A021012C3E522
:100F90004D94147026C3E54E94065003020E50C2C1
:100FA000AF901A0B740093D2AF7888F613C238C290
:100FB000394002D2384002D2398057C3E54D9415EA
:100FC0007038C3E54E9406404FC2AF901A0B7400C0
:100FD00093D2AFF8B801027402B802027401B803E8
:100FE000027404B8040274037888F613C238C23954
:100FF0004002D2384002D2398018C3E54D940C70BB
:1010000011755DA5755EF1C3E54E9406400A510069
:10101000D2AF754E00754D00755D00755E00C23033
:10102000020E50C2AF120ACFE4D2AFE4F559F52454
:10103000F525F53775590812046E1204EF30EDFDF1
:10104000A8BDA9BEE97001F8885A1204F3755908C1
:10105000C2AF12055A855856855857D2AF303A0755
:10106000C238303102D238D228753300120A1B122E
:101070000A441205691205991205691205991205AB
:101080006912082712092212097712059912081706
:10109000202C031204A9302C031204D912092212A5
:1010A00009A01205991208271209221209C912056E
:1010B000991208171209221209F21205991208272B
:1010C000120922120A1B1205991204EF12081712B4
:1010D0000922120A441204F3120599302827855870
:1010E0005679187A0CC3E53399400EC228D2298A62
:1010F00035855856855857800CC3E54F94014003F9
:10110000021081218B30291F202B1CE5351470061D
:10111000C229D22A0181F535203A07C3E54F94014F
:1011200040030210818064753600203A0F78FA7906
:10113000A4E760027803C3E55098504FE523604B65
:10114000303A17203805203107800F303102800AED
:10115000202B07D22B85585601B178F0302B05850E
:1011600058567820C3E571985003021081302B1B2C
:10117000C22BC238303102D238D229753512855887
:101180005601810536E54F6002218E753600C2AFEB
:10119000120ACF752500D2AF12047E120ACF752431
:1011A0000078A4E66006D287D291D293C3E5369444
:1011B000044003020C52020DE7901A0D78205139B9
:1011C000E520B4550AA35139E520B4AA028013756D
:1011D0005DA5755EF1120AE25100755D00755E0055
:1011E000801D901A0378807B0A5139A308DBFA909E
:1011F0001A0F788C7B1A5139A308DBFA901A29222E
:10120000C2AF517C5159901A007402513EA374032D
:10121000513EA37421513E901A0378807B0A513DC0
:10122000A308DBFA901A0F788C7B1A513DA308DBD8
:10123000FA518F516D901A2922E493F622E6438FDA
:1012400001538FFDFFC3E583941C400122EF855DB0
:10125000B7855EB7F0538FFE22438F02438F01851F
:101260005DB7855EB7901A0DF0538FFC22901A0D72
:101270007455513E901A0E74AA513E227A3079D09C
:101280007820901A405139E520F709A3DAF7227A3D
:101290003079D0901A40E7513E09A3DAF9227C0553
:0F12A00012045BDCFB22C2AF120A6CD2AF222217
:06148000544C5802030465
:10150000E4F52B757749757816757A10F57BF579C2
:10151000757CD885727D752B00E5E4A2E7B3E5E61E
:0815200092E0F5E60215B42289
:0315300002160B95
:1015500085817685D075E579857AD0857C81D25A6A
:08156000C077C07843E6802249
:10157000305A17C25A85D07AF579D078D0778581DC
:0B1580007C8576818575D085D77B3295
:1015B0000215DE32751CF6751DEB751EE07519BA45
:1015C000751AFEE573751B01B42812751CFC751D98
:1015D000F6751EF1751942751AFF751B0C22C2595A
:1015E000C572F452A4F44280C572C28CC28E758A50
:1015F00000758C007589AA851B8EC289C28BD2AA00
:10160000D2A8C2A9C2BBD28CC23432C2C0C0E030A0
:10161000592AD234E57D428042A4D0E07574A87581
:101620008921538EF0758BFF851A8C85198AC28D9E
:10163000C28FD2BBD28CD28E43A80A32D2AAD2A8F1
:10164000D0E0327B007A0180352059FD2034FA2029
:101650002906202803202000C2AFAB71AA70D2AFA8
:10166000EBC313FBEA13FAEBC313F9EA132AFAE903
:101670003BFBEA24FFEB34FF400474FFFBFAE4FC7D
:10168000C3EB136007FBEA13FA0C80F4EC234B5412
:101690000FC4FBEAC4FA540F4BFBEA54F0FA6BC4D4
:1016A0006B540F4A640FFA78A874E0C0E07416C057
:1016B000E0791C7D17EA540F242B83C0E0C015EAA3
:1016C000C4540F242083C0E0C015EB540F241683AC
:1016D000C0E0C015EBC4540F240B83C0E0C015223A
:1016E0007600D259C149000C1B24303F4B5766721B
:1016F0007C8693A2AFBC0000000000000000000048
:10170000E7F608A61C08A61E08791C22E7F608A61C
:101710001C08A61D08A61C08791C22E7F608A61EB0
:1017200008791D22E7F608A61E08A61C08791C22C7
:10173000E7F608A61C08A61C08A61D08791C22E7C7
:10174000F608A61D08A61D08791C22E7F608A61DA6
:1017500008A61C08791D22E7F608A61D08A61C0885
:10176000A61C08791C22E7F608A61C08A61D087905
:101770001D2209E7F608A61E08791C2209E7F608CB
:10178000A61D08791D2209E7F608A61D08A61C0853
:10179000791C22E7F608A61C08A61C08A61C0879D6
:1017A0001D2209E7F608A61C08A61D08791C2209B7
:1017B000E7F608A61C08A61C08791D2209E7F6080A
:0C17C000A61C08A61C08A61C08791C2208
:1019E0007597DE7597AD43EF02B4A5030219FD901C
:0A19F000FBFDE493B4A5F502FBC073
:1019FD00020BB7020321FFFFFFFFFFFF09FF01FFEE
:101A0D0055AA01FFFFFFFFFF03FFFFFF25D0285061
:0D1A1D0004FF02FF7AFF0701FFFF0000FF3A
:101A400023435F4C5F37302320202020202020209C
:101A500023424C48454C492445464D3842313023B9
:101A60002020202020202020202020202020202076
:101C0000C2AFC2D37597DE7597AD7581C075A90057
:101C100075A90043FF80752438752503B1DE752949
:101C2000A5752AF143F10153A4FED28075D4FF7546
:101C3000E3407DFA780379E67C1075220075230075
:101C4000901DEB7B06752498752501308002814B31
:101C5000208008D8FBD9F9DCF781BD308008D8FB9B
:101C6000D9F9DCF781BDB19EE493A3C39A6004DD8A
:101C7000C381BDDBDBB190600281347B08E493FA61
:101C8000A3B171DBF87A30B171752200752300B110
:101C900090EAFCEBFDC3ED94FE400EB1908A278BD9
:101CA00028ED30E0048A828B83B1907AC270D8C369
:101CB000ED94FE601950CEBD0029EC600F75200038
:101CC0007521FF752900752A000200008100A827F0
:101CD000A9280809D804D90281E0B194EAF281D494
:101CE0000D81A9C3ED94035051EDA2E092007AC595
:101CF000C3E5829400E583941C508C200010438F30
:101D000002438F018529B7852AB7F0300027A8271D
:101D1000A9280809438F01538FFDD804D902A135A2
:101D2000C3E583941C4003A3A11AE28529B7852A41
:101D3000B7F0A3A11A538FFC81857AC1BD030CE4CF
:101D400093A3FAB155DCF8B14D81858187AA22AB06
:101D500023B171EBFAEA6222752608C3E52313F575
:101D600023E52213F52250066323A0632201D52622
:101D7000EAB1DEB1DE75260AEAF4200102D2803033
:101D80000102C280B1DEC3134002C201D526EB229C
:101D9000B194EAFB208002A194308002A1997526BB
:101DA00008AE24AF25C3EF13FFEE13FEB1E2B1DEA0
:101DB000C3EA133080024480FA30E703632201C390
:101DC000E52313F523E52213F52250066323A063D0
:101DD0002201D526D9E52265236523F52222AE24EA
:101DE000AF250E0FDEFEDFFCD20122424C48656CAF
:091DF0006934373164E8B10601E1
:00000001FF
